:060000000200330217525A
:03000B0002175386
:0300130002177E53
:03001B0002177F4A
:0300230002178041
:03002B0002178138
:10003300759840758780758921758DFF758BFF7560
:100043008850D299758160758CFA758A0075A8827B
:100053007530007531007580FF75900075A00075CF
:10006300B03F782076FF08B830FA75F0FF7590003E
:10007300C2B77880E670257580FE75A00120A00FB9
:10008300300019C2007608901859121782800D208B
:10009300000AD200760890185C1217827881E67005
:1000A300257580FE75A00220A10F300119C20176CB
:1000B3000890185F121782800D20010AD20176087A
:1000C3009018621217827882E670257580FE75A0FB
:1000D3000420A20F300219C2027608901865121785
:1000E30082800D20020AD2027608901868121782C5
:1000F3007883E670257580FE75A00820A30F300372
:1001030019C203760890186B121782800D20030A18
:10011300D203760890186E1217827884E6702575DC
:1001230080FE75A01020A40F300419C20476089035
:100133001871121782800D20040AD20476089018D1
:10014300741217827885E670257580FE75A02020CD
:10015300A50F300519C2057608901877121782800B
:100163000D20050AD205760890187A121782788630
:10017300E670257580FE75A04020A60F300619C2D3
:1001830006760890187D121782800D20060AD20683
:1001930076089018801217827887E670257580FE9E
:1001A30075A08020A70F300719C20776089018831F
:1001B300121782800D20070AD2077608901886123C
:1001C30017827888E670257580FD75A00120A00F41
:1001D300300819C2087608901889121782800D20FA
:1001E300080AD208760890188C1217827889E6706C
:1001F300257580FD75A00220A10F300919C209766B
:100203000890188F121782800D20090AD2097608E8
:10021300901892121782788AE670257580FD75A072
:100223000420A20F300A19C20A76089018951217F3
:1002330082800D200A0AD20A760890189812178233
:10024300788BE670257580FD75A00820A30F300B11
:1002530019C20B760890189B121782800D200B0A87
:10026300D20B760890189E121782788CE67025754B
:1002730080FD75A01020A40F300C19C20C760890D5
:1002830018A1121782800D200C0AD20C7608901840
:10029300A4121782788DE670257580FD75A0202045
:1002A300A50F300D19C20D76089018A7121782807A
:1002B3000D200D0AD20D76089018AA121782788E97
:1002C300E670257580FD75A04020A60F300E19C27B
:1002D3000E76089018AD121782800D200E0AD20EEA
:1002E30076089018B0121782788FE670257580FD16
:1002F30075A08020A70F300F19C20F76089018B38E
:10030300121782800D200F0AD20F76089018B612AA
:1003130017827890E670257580FB75A00120A00FE9
:10032300301019C21076089018B9121782800D2068
:10033300100AD21076089018BC1217827891E670D2
:10034300257580FB75A00220A10F301119C211760B
:10035300089018BF121782800D20110AD211760857
:100363009018C21217827892E670257580FB75A0EB
:100373000420A20F301219C21276089018C5121762
:1003830082800D20120AD21276089018C8121782A2
:100393007893E670257580FB75A00820A30F3013B2
:1003A30019C21376089018CB121782800D20130AF6
:1003B300D21376089018CE1217827894E6702575BA
:1003C30080FB75A01020A40F301419C21476089076
:1003D30018D1121782800D20140AD21476089018AF
:1003E300D41217827895E670257580FB75A02020BE
:1003F300A50F301519C21576089018D712178280E9
:100403000D20150AD21576089018DA1217827896FD
:10041300E670257580FB75A04020A60F301619C223
:100423001676089018DD121782800D20160AD21650
:1004330076089018E01217827897E670257580FB8E
:1004430075A08020A70F301719C21776089018E3FC
:10045300121782800D20170AD21776089018E61219
:1004630017827898E670257580F775A00120A00F94
:10047300301819C21876089018E9121782800D20D7
:10048300180AD21876089018EC1217827899E67039
:10049300257580F775A00220A10F301919C21976AE
:1004A300089018EF121782800D20190AD2197608C6
:1004B3009018F2121782789AE670257580F775A066
:1004C3000420A20F301A19C21A76089018F51217D1
:1004D30082800D201A0AD21A76089018F812178211
:1004E300789BE670257580F775A00820A30F301B55
:1004F30019C21B76089018FB121782800D201B0A65
:10050300D21B76089018FE121782789CE670257528
:1005130080F775A01020A40F301C19C21C76089018
:100523001901121782800D201C0AD21C760890191B
:1005330004121782789DE670257580F775A0202038
:10054300A50F301D19C21D76089019071217828056
:100553000D201D0AD21D760890190A121782789E63
:10056300E670257580F775A04020A60F301E19C2CE
:100573001E760890190D121782800D201E0AD21EB6
:100583007608901910121782789FE670257580F708
:1005930075A08020A70F301F19C21F76089019136A
:1005A300121782800D201F0AD21F76089019161287
:1005B300178278A0E670257580EF75A00120A00F43
:1005C300302019C2207608901919121782800D2045
:1005D300200AD220760890191C12178278A1E6709F
:1005E300257580EF75A00220A10F302119C2217655
:1005F3000890191F121782800D20210AD221760834
:1006030090192212178278A2E670257580EF75A0E3
:100613000420A20F302219C222760890192512173E
:1006230082800D20220AD22276089019281217827E
:1006330078A3E670257580EF75A00820A30F3023FB
:1006430019C223760890192B121782800D20230AD2
:10065300D223760890192E12178278A4E670257596
:1006630080EF75A01020A40F302419C224760890BF
:100673001931121782800D20240AD224760890198A
:100683003412178278A5E670257580EF75A02020B7
:10069300A50F302519C225760890193712178280C5
:1006A3000D20250AD225760890193A12178278A6CA
:1006B300E670257580EF75A04020A60F302619C27D
:1006C30026760890193D121782800D20260AD2261D
:1006D300760890194012178278A7E670257580EF87
:1006E30075A08020A70F302719C2277608901943D9
:1006F300121782800D20270AD227760890194612F6
:10070300178278A8E670257580DF75A00120A00FF9
:10071300302819C2287608901949121782800D20B3
:10072300280AD228760890194C12178278A9E67005
:10073300257580DF75A00220A10F302919C2297603
:100743000890194F121782800D20290AD2297608A2
:1007530090195212178278AAE670257580DF75A06A
:100763000420A20F302A19C22A76089019551217AD
:1007730082800D202A0AD22A7608901958121782ED
:1007830078ABE670257580DF75A00820A30F302BAA
:1007930019C22B760890195B121782800D202B0A41
:1007A300D22B760890195E12178278ACE670257505
:1007B30080DF75A01020A40F302C19C22C7608906E
:1007C3001961121782800D202C0AD22C76089019F9
:1007D3006412178278ADE670257580DF75A020203E
:1007E300A50F302D19C22D76089019671217828034
:1007F3000D202D0AD22D760890196A12178278AE31
:10080300E670257580DF75A04020A60F302E19C233
:100813002E760890196D121782800D202E0AD22E83
:10082300760890197012178278AFE670257580DF0D
:1008330075A08020A70F302F19C22F760890197347
:10084300121782800D202F0AD22F76089019761264
:10085300178278B0E670257580BF75A00120A00FC0
:10086300303019C2307608901979121782800D2022
:10087300300AD230760890197C12178278B1E6706C
:10088300257580BF75A00220A10F303119C23176C2
:100893000890197F121782800D20310AD231760811
:1008A30090198212178278B2E670257580BF75A001
:1008B3000420A20F303219C232760890198512171C
:1008C30082800D20320AD23276089019881217825C
:1008D30078B3E670257580BF75A00820A30F303369
:1008E30019C233760890198B121782800D20330AB0
:1008F300D233760890198E12178278B4E670257574
:1009030080BF75A01020A40F303419C2347608902C
:100913001991121782800D20340AD2347608901967
:100923009412178278B5E670257580BF75A02020D4
:10093300A50F303519C235760890199712178280A2
:100943000D20350AD235760890199A12178278B697
:10095300E670257580BF75A04020A60F303619C2FA
:1009630036760890199D121782800D20360AD236EA
:1009730076089019A012178278B7E670257580BFA4
:1009830075A08020A70F303719C23776089019A3B6
:10099300121782800D20370AD23776089019A612D3
:1009A300178278B8E6702575807F75A00120A00FA7
:1009B300303819C23876089019A9121782800D2091
:1009C300380AD23876089019AC12178278B9E670D3
:1009D3002575807F75A00220A10F303919C23976A1
:1009E300089019AF121782800D20390AD239760880
:1009F3009019B212178278BAE6702575807F75A0B8
:100A03000420A20F303A19C23A76089019B512178A
:100A130082800D203A0AD23A76089019B8121782CA
:100A230078BBE6702575807F75A00820A30F303B47
:100A330019C23B76089019BB121782800D203B0A1E
:100A4300D23B76089019BE12178278BCE6702575E2
:100A5300807F75A01020A40F303C19C23C7608900B
:100A630019C1121782800D203C0AD23C76089019D6
:100A7300C412178278BDE6702575807F75A020208B
:100A8300A50F303D19C23D76089019C71217828011
:100A93000D203D0AD23D76089019CA12178278BEFE
:100AA300E6702575807F75A04020A60F303E19C2E1
:100AB3003E76089019CD121782800D203E0AD23E51
:100AC30076089019D012178278BFE6702575807F5B
:100AD30075A08020A70F303F19C23F76089019D325
:100AE300121782800D203F0AD23F76089019D61242
:100AF300178275A000C2B778C0E670257580FE75B1
:100B0300900120900F304019C24076089019D912F5
:100B13001782800D20400AD24076089019DC121704
:100B23008278C1E670257580FE75900220910F30A2
:100B33004119C24176089019DF121782800D2041B6
:100B43000AD24176089019E212178278C2E670251C
:100B53007580FE75900420920F304219C2427608C8
:100B63009019E5121782800D20420AD2427608902E
:100B730019E812178278C3E670257580FE75900810
:100B830020930F304319C24376089019EB12178252
:100B9300800D20430AD24376089019EE121782780B
:100BA300C4E670257580FE75901020940F304419AB
:100BB300C24476089019F1121782800D20440AD29C
:100BC3004476089019F412178278C5E6702575806B
:100BD300FE75902020950F304519C245760890196F
:100BE300F7121782800D20450AD24576089019FA2C
:100BF30012178278C6E670257580FE7590402096A0
:100C03000F304619C24676089019FD121782800DDF
:100C130020460AD2467608901A0012178278C7E651
:100C230070257580FE75908020970F304719C24755
:100C33007608901A03121782800D20470AD247764E
:100C430008901A0612178278C8E670257580FD751C
:100C5300900120900F304819C2487608901A091263
:100C63001782800D20480AD2487608901A0C121772
:100C73008278C9E670257580FD75900220910F304A
:100C83004919C2497608901A0F121782800D20491C
:100C93000AD2497608901A1212178278CAE670258A
:100CA3007580FD75900420920F304A19C24A760868
:100CB300901A15121782800D204A0AD24A7608909C
:100CC3001A1812178278CBE670257580FD75900887
:100CD30020930F304B19C24B7608901A1B121782C0
:100CE300800D204B0AD24B7608901A1E1217827879
:100CF300CCE670257580FD75901020940F304C194B
:100D0300C24C7608901A21121782800D204C0AD209
:100D13004C7608901A2412178278CDE670257580D8
:100D2300FD75902020950F304D19C24D7608901A0D
:100D330027121782800D204D0AD24D7608901A2A69
:100D430012178278CEE670257580FD759040209647
:100D53000F304E19C24E7608901A2D121782800D4D
:100D6300204E0AD24E7608901A3012178278CFE6B8
:100D730070257580FD75908020970F304F19C24FF5
:100D83007608901A33121782800D204F0AD24F76BD
:100D930008901A3612178278D0E670257580FB7595
:100DA300900120900F305019C2507608901A3912D2
:100DB3001782800D20500AD2507608901A3C1217E1
:100DC3008278D1E670257580FB75900220910F30F3
:100DD3005119C2517608901A3F121782800D205183
:100DE3000AD2517608901A4212178278D2E67025F9
:100DF3007580FB75900420920F305219C252760809
:100E0300901A45121782800D20520AD2527608900A
:100E13001A4812178278D3E670257580FB759008FF
:100E230020930F305319C2537608901A4B1217822E
:100E3300800D20530AD2537608901A4E12178278E7
:100E4300D4E670257580FB75901020940F305419EB
:100E5300C2547608901A51121782800D20540AD278
:100E6300547608901A5412178278D5E67025758047
:100E7300FB75902020950F305519C2557608901AAE
:100E830057121782800D20550AD2557608901A5AA8
:100E930012178278D6E670257580FB7590402096F0
:100EA3000F305619C2567608901A5D121782800DBC
:100EB30020560AD2567608901A6012178278D7E61F
:100EC30070257580FB75908020970F305719C25796
:100ED3007608901A63121782800D20570AD257762C
:100EE30008901A6612178278D8E670257580F77510
:100EF300900120900F305819C2587608901A691241
:100F03001782800D20580AD2587608901A6C12174F
:100F13008278D9E670257580F775900220910F309D
:100F23005919C2597608901A6F121782800D2059E9
:100F33000AD2597608901A7212178278DAE6702567
:100F43007580F775900420920F305A19C25A7608AB
:100F5300901A75121782800D205A0AD25A76089079
:100F63001A7812178278DBE670257580F77590087A
:100F730020930F305B19C25B7608901A7B1217829D
:100F8300800D205B0AD25B7608901A7E1217827856
:100F9300DCE670257580F775901020940F305C198E
:100FA300C25C7608901A81121782800D205C0AD2E7
:100FB3005C7608901A8412178278DDE670257580B6
:100FC300F775902020950F305D19C25D7608901A51
:100FD30087121782800D205D0AD25D7608901A8AE7
:100FE30012178278DEE670257580F775904020969B
:100FF3000F305E19C25E7608901A8D121782800D2B
:10100300205E0AD25E7608901A9012178278DFE685
:1010130070257580F775908020970F305F19C25F38
:101023007608901A93121782800D205F0AD25F769A
:1010330008901A9612178278E0E670257580EF758E
:10104300900120900F306019C2607608901A9912AF
:101053001782800D20600AD2607608901A9C1217BE
:101063008278E1E670257580EF75900220910F304C
:101073006119C2617608901A9F121782800D206150
:101083000AD2617608901AA212178278E2E67025D6
:101093007580EF75900420920F306219C262760852
:1010A300901AA5121782800D20620AD262760890E8
:1010B3001AA812178278E3E670257580EF759008F9
:1010C30020930F306319C2637608901AAB1217820C
:1010D300800D20630AD2637608901AAE12178278C5
:1010E300E4E670257580EF75901020940F30641935
:1010F300C2647608901AB1121782800D20640AD256
:10110300647608901AB412178278E5E67025758024
:10111300EF75902020950F306519C2657608901AF7
:10112300B7121782800D20650AD2657608901ABA25
:1011330012178278E6E670257580EF759040209649
:101143000F306619C2667608901ABD121782800D99
:1011530020660AD2667608901AC012178278E7E6EC
:1011630070257580EF75908020970F306719C267DF
:101173007608901AC3121782800D20670AD2677609
:1011830008901AC612178278E8E670257580DF7515
:10119300900120900F306819C2687608901AC9121E
:1011A3001782800D20680AD2687608901ACC12172D
:1011B3008278E9E670257580DF75900220910F3003
:1011C3006919C2697608901ACF121782800D2069B7
:1011D3000AD2697608901AD212178278EAE6702545
:1011E3007580DF75900420920F306A19C26A760801
:1011F300901AD5121782800D206A0AD26A76089057
:101203001AD812178278EBE670257580DF7590087F
:1012130020930F306B19C26B7608901ADB1217827A
:10122300800D206B0AD26B7608901ADE1217827833
:10123300ECE670257580DF75901020940F306C19E3
:10124300C26C7608901AE1121782800D206C0AD2C4
:101253006C7608901AE412178278EDE67025758093
:10126300DF75902020950F306D19C26D7608901AA6
:10127300E7121782800D206D0AD26D7608901AEA64
:1012830012178278EEE670257580DF759040209600
:101293000F306E19C26E7608901AED121782800D08
:1012A300206E0AD26E7608901AF012178278EFE653
:1012B30070257580DF75908020970F306F19C26F8E
:1012C3007608901AF3121782800D206F0AD26F7678
:1012D30008901AF612178278F0E670257580BF75AC
:1012E300900120900F307019C2707608901AF9128D
:1012F3001782800D20700AD2707608901AFC12179C
:101303008278F1E670257580BF75900220910F30C9
:101313007119C2717608901AFF121782800D20711D
:101323000AD2717608901B0212178278F2E67025B2
:101333007580BF75900420920F307219C2727608BF
:10134300901B05121782800D20720AD272760890C4
:101353001B0812178278F3E670257580BF75900815
:1013630020930F307319C2737608901B0B121782E8
:10137300800D20730AD2737608901B0E12178278A1
:10138300F4E670257580BF75901020940F307419A2
:10139300C2747608901B11121782800D20740AD232
:1013A300747608901B1412178278F5E67025758001
:1013B300BF75902020950F307519C2757608901B64
:1013C30017121782800D20750AD2757608901B1AA2
:1013D30012178278F6E670257580BF7590402096C7
:1013E3000F307619C2767608901B1D121782800D76
:1013F30020760AD2767608901B2012178278F7E6B9
:1014030070257580BF75908020970F307719C2774C
:101413007608901B23121782800D20770AD27776E5
:1014230008901B2612178278F8E6702575807F7561
:10143300900120900F307819C2787608901B2912FA
:101443001782800D20780AD2787608901B2C121709
:101453008278F9E6702575807F75900220910F30B0
:101463007919C2797608901B2F121782800D207983
:101473000AD2797608901B3212178278FAE6702521
:1014830075807F75900420920F307A19C27A76089E
:10149300901B35121782800D207A0AD27A76089033
:1014A3001B3812178278FBE6702575807F759008CC
:1014B30020930F307B19C27B7608901B3B12178257
:1014C300800D207B0AD27B7608901B3E1217827810
:1014D300FCE6702575807F75901020940F307C1981
:1014E300C27C7608901B41121782800D207C0AD2A1
:1014F3007C7608901B4412178278FDE67025758070
:101503007F75902020950F307D19C27D7608901B42
:1015130047121782800D207D0AD27D7608901B4AE0
:1015230012178278FEE6702575807F7590402096AD
:101533000F307E19C27E7608901B4D121782800DE4
:10154300207E0AD27E7608901B5012178278FFE61F
:10155300702575807F75908020970F307F19C27F2B
:101563007608901B53121782800D207F0AD27F7654
:1015730008901B5612178275A0007590007840E6FC
:1015830070247580FED2B720B70F30F019C2F07601
:1015930008901829121782800D20F00AD2F07608DD
:1015A30090182C1217827841E670247580FDD2B70B
:1015B30020B70F30F119C2F1760890182F12178255
:1015C300800D20F10AD2F176089018321217827832
:1015D30042E670247580FBD2B720B70F30F219C2F0
:1015E300F27608901835121782800D20F20AD2F293
:1015F30076089018381217827843E670247580F7BE
:10160300D2B720B70F30F319C2F3760890183B1204
:101613001782800D20F30AD2F3760890183E121732
:10162300827844E670247580EFD2B720B70F30F488
:1016330019C2F47608901841121782800D20F40A1B
:10164300D2F476089018441217827845E670247510
:1016530080DFD2B720B70F30F519C2F5760890189E
:1016630047121782800D20F50AD2F5760890184AA2
:101673001217827846E670247580BFD2B720B70F61
:1016830030F619C2F6760890184D121782800D2095
:10169300F60AD2F676089018501217827847E67049
:1016A3002475807FD2B720B70F30F719C2F77608B9
:1016B300901853121782800D20F70AD2F7760890FC
:1016C3001856121782D2B220B21C7532071217B500
:1016D3001217A7D532067532011217B51217AED2FB
:1016E300B220B20280EDD2B320B31C7532071217B9
:1016F300D21217A7D532067532011217D21217AEBE
:10170300D2B320B30280EDD2B420B41C75320712D9
:1017130017EF1217A7D532067532011217EF1217FA
:10172300AED2B420B40280EDD2B520B51C75320719
:1017330012180C1217A7D5320675320112180C12A3
:1017430017AED2B520B50280ED020070020033322D
:10175300C0D0C0E0C000D53304C2B0D2B67880E6B2
:1017630060011608B800F87840E660011608B8482A
:10177300F8758CFAD000D0E0D0D0323232323275E4
:101783003310D2B0C2B6E4933099FDC299F599A350
:10179300E4933099FDC299F599A3E4933099FDC27E
:1017A30099F599227E20DFFEDEFC227E60DFFEDEDD
:1017B300FC22753320D2B0C2B63099FDC299759917
:1017C300C03099FDC2990530E530547FF5992275F3
:1017D3003320D2B0C2B63099FDC2997599C0309901
:1017E300FDC2991530E530547FF59922753320D227
:1017F300B0C2B63099FDC2997599C13099FDC299AD
:101803000531E531547FF59922753320D2B0C2B644
:101813003099FDC2997599C13099FDC2991531E589
:1018230031547FF59922B0407FB04000B0437FB080
:101833004300B0017FB00100B0027FB00200B140AD
:101843007FB14000B1437FB14300B1017FB10100DB
:10185300B1027FB102009024408024009025408093
:10186300250090264080260090274080270090285E
:1018730040802800902940802900902A40802A0037
:10188300902B40802B00902C40802C00902D40808A
:101893002D00902E40802E00902F40802F009030FE
:1018A30040803000903140803100903240803200DF
:1018B3009033408033009034408034009035408032
:1018C300350090364080360090374080370090389E
:1018D30040803800903940803900903A40803A0087
:1018E300903B40803B00903C40803C00903D4080DA
:1018F3003D00903E40803E00903F40803F0090403E
:10190300408040009041408041009042408042002E
:101913009043408043009044408044009045408081
:1019230045009046408046009047408047009048DD
:1019330040804800904940804900904A40804A00D6
:10194300904B40804B00904C40804C00904D408029
:101953004D00904E40804E00904F40804F0090507D
:10196300408050009051408051009052408052007E
:101973009053408053009054408054009124408100
:10198300240091254081250091264081260091273E
:101993004081270091284081280091294081290016
:1019A300912A40812A00912B40812B00912C408168
:1019B3002C00912D40812D00912E40812E00912FDE
:1019C30040812F00913040813000913140813100BE
:1019D3009132408132009133408133009134408110
:1019E300340091354081350091364081360091377E
:1019F3004081370091384081380091394081390066
:101A0300913A40813A00913B40813B00913C4081B7
:101A13003C00913D40813D00913E40813E00913F1D
:101A230040813F009140408140009141408141000D
:101A3300914240814200914340814300914440815F
:101A430044009145408145009146408146009147BD
:101A530040814700914840814800914940814900B5
:101A6300914A40814A00914B40814B00914C408107
:101A73004C00914D40814D00914E40814E00914F5D
:101A830040814F009150408150009151408151005D
:101A930091524081520091534081530091544081AF
:101AA3005400921840821800921940821900921A29
:101AB30040821A00921B40821B00921C40821C0031
:101AC300921D40821D00921E40821E00921F408282
:101AD3001F00922040822000922140822100922206
:101AE30040822200922340822300922440822400D9
:101AF300922540822500922640822600922740822A
:101B03002700922840822800922940822900922AA5
:101B130040822A00922B40822B00922C40822C0080
:101B2300922D40822D00922E40822E00922F4082D1
:101B33002F00923040823000923140823100923245
:101B43004082320092334082330092344082340028
:101B5300923540823500204D757A796B616E742021
:101B6300332076312E306620323030362D31312D10
:101B73003234202863294164616D20536D69616C9F
:101B8300656B206A616E6B6F6D757A796B616E74CC
:101B93004077702E706C207777772E736D69616C48
:101BA300656B2E7072762E706C2057737A656C6B32
:101BB3006965207072617761207A617374727A65E6
:101BC3007A6F6E652E204A616B69656B6F6C7769FE
:101BD300656B207A6173746F736F77616E696120CF
:101BE3006B6F6D657263796A6E65206B6F647520C8
:101BF3006E6965646F7A776F6C6F6E652E20416CCA
:101C03006C205269676874732052657365727665D8
:101C1300642E204672656520666F72206E6F6E209B
:101C2300636F6D6D65726369616C206F6E6C792E85
:011C33002090
:00000001FF
